:0300000002020FEA
:03000B0002064F9B
:03004300020100B7
:030033000201586F
:10010000020652000206D3000206D300020699003E
:100110000206BD000206D3000206D3000206D30089
:100120000206D3000206D3000206D3000206D30063
:100130000206D3000206D3000206D3000206D30053
:100140000206D3000206D3000206D3000206D30043
:100150000206D3000206D30053D8EF32907FC8E0E6
:1001600020E15C200B5990784F747DF0A374C0F0AF
:10017000907FC9E0F8907854F0907851B41F0A74D9
:100180000FF0A37496F002019674D5254EF9741001
:10019000354FF0A3E9F0907855F0E8B41F22D2076C
:1001A000754E00754F007550007551007552007501
:1001B0005300907855E030E7F9907FC9F0809D2298
:1001C000F9E54E29F54EF8E54F3400F54FB4070A2E
:1001D000E8B40006754E00754F00E92552F9F55256
:1001E00074003553F553C92440C93400F87400C372
:1001F0009974079850BCD20B7954E72401F709E7AA
:100200003400F709E73400F709E73400F780A375F5
:10021000815F1209411202ABE41209A34005D20C1E
:1002200012090E12033030060312035D300405007C
:100230000000C20430080512082A80EA315C300749
:100240000D1208C6907FC9F0300703120705E55B61
:1002500054046558604E6558F558E55A703BD559B9
:1002600043755910200C0BE41209A34037D20C023D
:1002700002A4E533120993600612099F0202A4C288
:100280000C900F0A7400F0A3F0900F2074FFF0A3FD
:03029000F0A3F0E8
:100293001203300202A4D55A087400120B53120938
:1002A3009F00000000004126C206C204C205C2002E
:1002B300C201755A00755800755910C20C74FF902D
:1002C3007FABF0907FA9F0907FAAF0754055754100
:1002D3005375424275435375570075540075550065
:1002E300755600C20BC207C208D2E843D820538E0A
:1002F300F85391EF907F92E054FDF0907FAFE0448C
:1003030011F0907FAEE04409F0907FDE7405F09029
:100313007FDF7405F0907FDD7409F0D2AF907FD654
:10032300E04402F0758901758810D2A922907FD626
:10033300E04408F0F0E04402F07FDC7E031206376D
:10034300907FD6E054F7F07E037FFF780112061EFC
:10035300200606DFF6DEF480D422907FE9E0700BFE
:10036300907FE8E024DF70000203A8147003020406
:100373001424FE700302046F24FB70030204E114CF
:1003830070030204F214700302050E1470030205D5
:100393001D240570030205AA907FE8E030E60302FE
:1003A30005320205EE907FE8E0247F60231460307D
:1003B3002402705AA205E43325E0FFA200E4334F80
:1003C300907F00F0E4A3F0907FB57402F00205F58E
:1003D300E4907F00F0A3F0907FB57402F00205F57E
:1003E300907FECE0F45480C4FFE0540720010270D6
:0B03F3001D2F25E024B4F58275837FE8
:1003FE00E054FE907F00F0E4A3F0907FB57402F01D
:10040E000205F50205EE907FE8E024FE6007240267
:10041E0060400205EE907FEAE07043907FECE0F4DE
:10042E005480C4FFE0540720010270322F25E024CF
:10043E00B4F58275837FE4F0907FECE05480131363
:10044E0013541FFFE054072F907FD7F0D2E5F00230
:10045E0005F5907FEAE0B40105C2050205F5020537
:10046E00EE907FE824FE6007240260580205F590A6
:10047E007FEAE0705B907FECE0F45480C4FFE054C0
:10048E000720010270D82F25E024B4F58275837FF2
:10049E007401F0C083C082907FECE054801313137C
:1004AE00541FFFE054072F907FD7F0D2E5F0D08293
:1004BE00D083EF20E407A37401F00205F5E0D2E14A
:1004CE00F00205F5907FEAE0B40105D2050205F5CC
:1004DE000205EE907F00E4A20133F0907FB5740127
:1004EE00F00205F5907FEAE0600BB40110D2011224
:1004FE0005FF0205F5C2011205FF0205F50205EE24
:10050E00907F00E530F0907FB57401F00205F52084
:10051E00010302052F907FEAE0F5301205FF020578
:10052E00F50205EE907FE9E0B410257400300C0F53
:10053E00907FECE0F9C3E5339974004002E5349006
:10054E007F00F0A3E533F0907FB57402F00205F55D
:10055E00B41146907FECE0B53332E55A7012E533B4
:10056E0012099360277403120B53755A04120B660B
:10057E00120B83E4907C407D40C0E0120C5FEFF0E4
:10058E00A3EEF0A3D0E004DDF0120B8A907FD474BA
:10059E007CF0A37440F00205F50205F5907FEBE0C8
:1005AE0024FE601414601E24027035907FD4740FE4
:1005BE00F0A37400F00205F5907FD4740FF0A374CD
:1005CE0012F00205F5907FEAE023F9900F3293C9FD
:1005DE000493C9907FD4F0A3E9F00205F50205F566
:1005EE00907FB4E04401F0907FB4E04402F0C20684
:1005FE0022907FD7E47F08F0D2E5F0C2E505E0DF78
:10060E00F67F087410F0D2E5F0C2E505E0DFF622C1
:10061E00C082C083C0E090FB4BA3E582458370F996
:10062E00D8F4D0E0D083D082228E318F32E53215CD
:10063E0032AE31700215314E60067801D11E80ED5A
:10064E0022055B32C0E0C083C082C085C084C086F4
:10065E00C0D074EF5291907FAB7401F0907FE8E0C0
:10066E00B42117A3E0B4FF121206D412093B758110
:10067E005F51CEB1F51206984126D206D0D0D08663
:10068E00D084D085D082D083D0E032C0E0C083C089
:10069E00825391EF907FAB7408F0907FD6E0448048
:0A06AE00F0D2040000000000D0822A
:1006B800D083D0E032C0E0C083C0825391EF907FF6
:1006C800AB7410F0D082D083D0E03232300C2DE5FC
:1006D8005A60297407120A8724B06020740E790CB6
:1006E800120A8ED11E740E7908120A8E78007900CB
:1006F8007407120A8730E704D9F6D8F422754D003A
:10070800300C0BE55A702BE5331209937005740110
:100718000207E27403120B53120B66315C740679FC
:10072800A0120A8E74017900120A8E740E790812CA
:100738000A8E755A04120938315C7407120A8754F4
:100748008870F5740479FF120A8E740579FF120A0D
:100758008E740779A0120A8E315C7407120A8754C6
:100768000860F5315C7407120A87548070F57E06BC
:100778007F00900FA5E0B41203000000120B263191
:100788005C120B4160F97407120A877402120A8717
:100798005403700A12084B315C120DA780E11470E3
:1007A8000574020207E214702530091A7404120A4B
:1007B80087FC7405120A87FD7F00120AADDCF980F8
:1007C800BE74020207E212084B120D0180B17407D1
:1007D800120A8754016003000000F54C300A192002
:1007E8000903120885E54D6031907FB923F0907FA9
:1007F800B8E020E1F902082220091FAD48AC4912EF
:10080800015CA952A853755200755300C20BEDC381
:1008180099FDEC98FC40034D70E5D208C207120818
:100828002A22907FB8E054037018C208907E00799D
:10083800407F0DE7F009A3DFFA907FB9740DF0123D
:10084800093B227404120A87FC7405120A87FDD238
:0C0858000975F0007948E7C39C42F0F7F6
:1008640009E79D42F0F709E7940042F0F709E7949D
:100874000042F0F7E5F06002C209EDC313CC13FDAA
:10088400227948E754C0094709470947601F7C009B
:100894007D20120D017948E7C39440F709E79400DD
:1008A400F709E79400F709E79400F780D4E5485482
:1008B4003F600E7C00C313FD74003400F548120D34
:1008C4000122907FE3740FF0A37496F0A3E0B45573
:1008D40028E0B45324E0B44220E0B4431C79447FBC
:1008E40004E0F709DFFB7F04D209E0F76002C209E4
:1008F40009DFF7E0A2E7920A22C207907FB8E0443A
:1009040001F0907FC8E04401F022E53312099360BE
:1009140022120B837437900F867D04C0E0120C5FA3
:10092400EFF0A3A3EEF0A3A3D0E004DDEE120B8A54
:0409340012099F22E3
:10093800D28522C28522B2852290784A7480F090AE
:100948007827743FF0907826743FF0907849E0D289
:10095800E0F0907F947400F075B3FF75B4F075B251
:100968002012093B2275B440907826743FF09078A5
:10097800277400F090784A748AF02290784A74803C
:0B098800F0907827743FF075B4F02267
:10099300F5331209C174004002740122120A1422B1
:1009A300F533120A141209C150080533E53370F503
:1009B300D322120AA5F53412099FE533C322E53386
:1009C300F4F59075A0F0120A0FF4F590120A0FB225
:1009D300A7120A0FB2A7120A0FB2A7120A0FC2A5D3
:1009E300E533540765A054077020D2A5E533F454CA
:1009F3000765A054077013D2A7C0017910740412BD
:100A03000A9DD001C3E533020A0ED322C001D001EF
:100A130022C2A7120A0F75A00022C2A4F590120ADF
:100A23000FB2A522C2A4F590B2A622D2A475B30038
:100A3300B2A6120A0FE590C2A475B3FF22D2A40591
:100A430086E583907FE3F0E582A3F0A375B300B25C
:100A5300A61F120A0FE590F0B2A6DFF6120A0FE501
:100A630090F0C2A475B3FF058622C2A40586E58370
:100A7300907FE3F0E582A3F0A3E0F59000B2A6DF58
:100A8300F80586224440120A1D80A04440120A1D24
:100A9300E980914400120A1D80914400120A1DE965
:100AA3008082740B120A96543F2279507404120AFE
:100AB3009DEF4440120A1D120A2ECF4440120A1D14
:100AC300120A2EFE79107404120A9D2279507404BE
:100AD300120A9DEF4440120A1DED120A27EF44400B
:100AE300120A1DEE120A2779107404120A9D22EECF
:020AF30023FEE0
:100AF500E534B405127438120A1DEE120A27740083
:100B0500120A2774104FFF79507404120A9DEF449E
:100B150040120A1DEEFF120A4079107404120A9D54
:100B25002279507404120A9DEF4440120A1DEE23E7
:100B3500FF120A6D79107404120A9D22740B120AB1
:100B4500965480227405120A9654C0232322540316
:100B55000303F97405120A96543F49F97405020A0C
:100B65009D7405120A964408F97405020A9D7406D7
:100B7500020A96C0E0F97406120A9DD0E022120B13
:100B850073440880EE120B7354F780E7120B73441D
:100B95000480E0120B7354FB80D9120B91120BCE1B
:100BA50060FB80EFC0E0C0F0540160027402F5F014
:100BB500120B7354FC45F0120B784401120B785458
:100BC500FE120B78D0F0D0E0227400120A96548001
:100BD5006002740122120B917401120BA914120BFD
:100BE500A9120BA904120BA9120BA9120BA9120B1E
:100BF500A9120BA9120BA9120B9822120B917401C1
:100C0500120BA914120BA9120BA9120BA9120BA9ED
:100C1500120BA9120BA9120BA9120BA9120B9822E0
:100C2500C0E0120B917401120BA97400120BA97488
:100C350001120BA9D0E02323237B06120BA923DB8A
:100C4500FAEE7B0823120BA9DBFAEF7B0823120BC4
:100C5500A9DBFA120B98120B9F22C0E0120B9174BC
:0F0C650001120BA9120BA914120BA9D0E0232323
:100C7400237B06120BA923DBFA7B08C0E074001265
:100C84000BA9120BCE13D0E033DBF0FE7B08C0E0DF
:100C94007400120BA9120BCE13D0E033DBF0FF1259
:100CA4000B9822120B917401120BA914120BA912A6
:100CB4000BA904120BA914120BA9120BA9120BA94C
:100CC400120BA9120BA9120B98120B9F120B917401
:100CD40001120BA914120BA9120BA9120BA90412CD
:100CE4000BA9120BA9120BA9120BA9120BA97B10A9
:100CF40014120BA9DBFB120B98120B9F22E534B4E0
:100D040005137438120A1DEDC333FEEC33CE120AF8
:100D140027EE120A2779507404120A9D7440A934EC
:100D2400B905024410120A1DD2A475B300907FE3E2
:100D3400747EF0ED4C605F907FE47400254D254D8A
:100D4400F07420C3954DF9EDC399FDEC9400FCE9D2
:100D54005006E92D7C007D00FF254DF54DC0E0B225
:100D6400A6907FB8E020E1FC907FE5DF02800FE5EC
:100D740090B2A6F000E590B2A6F00000DFF1E59095
:100D8400B2A6F000E590F0D0E0B420A7907FB9239C
:100D9400F0754D00809DC2A475B3FF7910740412E0
:100DA4000A9D22EDC333FDEC33FC79507404120A1E
:100DB4009D7440120A1D12015CED4C700879107488
:100DC40004120A9D22907FE474D52550F0907FE3AD
:100DD40074103551F012015CA853A952E84960F52A
:100DE400E9C39DE89C4004EDF9ECF8E92550FBE8E3
:100DF4003551FA7400C39BFF74079AFE40064F7086
:100E040013020E14EB2FFBEA3EFAE92FF9E83EF841
:100E14007A007B008B508A51C3E55299F552E55311
:100E240098F553907FE5E8C313FAE913FBEAC3137B
:100E3400FAEB13FB500AE0F590B2A6E0F590B2A6E7
:100E4400EAC313FAEB13FB5014E0F590B2A6E0F5F5
:100E540090B2A6E0F590B2A6E0F590B2A6EAC3136C
:100E6400FAEB13FB5028E0F590B2A6E0F590B2A699
:100E7400E0F590B2A6E0F590B2A6E0F590B2A6E057
:100E8400F590B2A6E0F590B2A6E0F590B2A6EB60BC
:100E940052E0F590B2A6E0F590B2A6E0F590B2A6C5
:100EA400E0F590B2A6E0F590B2A6E0F590B2A6E027
:100EB400F590B2A6E0F590B2A6E0F590B2A6E0F502
:100EC40090B2A6E0F590B2A6E0F590B2A6E0F59057
:0C0ED400B2A6E0F590B2A6E0F590B2A640
:100EE000E0F590B2A6DBAEEDC399FDEC98FC300BBB
:100EF0000CE9C39440E50094004002C20B020DBA15
:100F00001201100100000040C90AFF10060301028F
:100F10000301090220000101004000090400000251
:100F20000802500007058202400000070502024047
:100F300000000F3A0F3E0F5E0F84040309042003E4
:100F40004D006900630072006F00200053006F00C5
:100F50006C007500740069006F006E00730026035A
:100F60004200410043004B005000410043004B0051
:100F70002000550053004200200043006100620041
:100F80006C0065001203300030003000300030008B
:060F9000300030003000CB
:00000001FF
